:1000000025C19EC23EC13DC13CC13BC13AC139C1BF
:1000100038C137C136C135C134C133C132C131C134
:1000200030C12FC12EC12DC12CC12BC12AC129C164
:1000300028C127C10403090418037200610070007D
:1000400068006E00650074002E006E00650074008C
:100050000A03310030003000300005010905A1011C
:100060000901A10009300931150026FF0075089526
:10007000028102C005091901290815002501750131
:1000800095088102C005010902A1010901A100052D
:1000900009190129021500250195027501810295B2
:1000A00001750681030501093009311581257F7528
:1000B0000895028106C0C0120101010000000881FC
:1000C00017970A08010102030105010905A10109A9
:1000D00001A10009300931150026FF0075089502BD
:1000E0008102C00509190129041500250175019532
:1000F000048102750195048103C012010101000011
:1001000000088117990A080101000001050109058D
:10011000A1010901A10009300931150026FF007570
:100120000895028102C00509190129081500250159
:10013000750195088102C0120101010000000881CB
:1001400017960A08010102030112010101000000D3
:100150000840177A0508010102030105010905A1FC
:10016000010901A10009300931150026FF007508B9
:1001700095028102C005091901290815002501759C
:100180000195088102C005010904A1010901A1002E
:10019000850109300931150026FF00750895028197
:1001A0000205091901290815002501750195088125
:1001B00002C0C005010904A1010901A100850209CD
:1001C000300931150026FF007508950281020509E6
:1001D0001901290815002501750195088102C0C083
:1001E00005010904A1010901A100850309300931B4
:1001F000150026FF007508950281020509190129DD
:100200000815002501750195088102C0C005010986
:1002100004A1010901A10085040930093115002656
:10022000FF007508950281020509190129081500CA
:100230002501750195088102C0C01201010100006D
:10024000000881179D0A08010102030111241FBE45
:10025000CFEFD4E0DEBFCDBF12E0A0E0B1E0E8E731
:10026000FBE102C005900D92A833B107D9F712E067
:10027000A8E3B2E001C01D92A83CB107E1F740D36A
:1002800079CCBECEE9E6F0E0808183608083E89A95
:1002900083EC80939E0208950F931F93CF93DF9377
:1002A0009091AE0219160CF0AFC02091AB02809174
:1002B000AA028D3209F09EC08AE5809301019B302D
:1002C00009F098C0CCE0D0E0C21BD109CE54DD4F7C
:1002D0008881807609F080C010929C0289818823F1
:1002E00059F410929D028CE992E09093AD028093B4
:1002F000AC0230E822E077C0853021F48A81809317
:10030000AF0268C0863009F04AC08B81813009F4A1
:1003100041C0823019F4CE0176D260C0833069F5D5
:100320008A81882349F484E390E09093AD0280931E
:10033000AC0230EC24E057C0813049F488E390E00F
:100340009093AD028093AC0230EC28E14CC0823037
:1003500049F483E091E09093AD028093AC0230E8E1
:1003600028E341C08330E9F580E590E09093AD0249
:100370008093AC0230EC2CE036C0813249F48BE43F
:1003800092E09093AD028093AC0230EC29E02BC058
:10039000823239F5CE0137D2282F30EC24C0883094
:1003A00019F481EB92E00AC0893021F48A818093AC
:1003B000B10210C08A3049F48CE992E09093AD020A
:1003C0008093AC0230E821E00EC08B3019F483EC4E
:1003D00080939E0230E806C0CE0143D2282F30E839
:1003E00002C030EC20E08F81882339F48E8182179F
:1003F00028F003C030E880E001C0822F309338023B
:10040000809300011092AE028091010184FF49C0E7
:10041000809100018F3F09F444C0182F893008F003
:1004200018E0811B809300018091380280FD02C09A
:100430000BE401C003EC8F5F809338022091AC0283
:100440003091AD0286FD05C0D901912FE4E9F2E0BB
:1004500011C0A4E9B2E080E090E006C0F901E80F25
:10046000F91FE491ED9301961817C1F705C08D911E
:10047000819391509923D9F7F901E10FF11DF09380
:10048000AD02E093AC0284E992E0612F55D01830C0
:1004900019F08FEF80930001009393021C5F10937B
:1004A00001019AE089B1857031F49150D9F7109229
:1004B000AF021092A902DF91CF911F910F91089581
:1004C0001F93DC01162F8091020184FF0AC08091E6
:1004D0009E0298E8892780939E02912FEFE9F2E02F
:1004E00007C08AE580930201F8CF8D9181939150E6
:1004F0009923D9F78FE992E0612F1ED01C5F1093EA
:1005000002011F910895A82FB92F8FEF9FEF41E0AF
:1005100050EA615070F02D9138E0722F782796954F
:100520008795269570FF02C0842795273A95A9F7ED
:10053000F0CF809590950895E6DF8D939D93089573
:10054000CF93CFB7CF93489BFECF489B09C0489B22
:1005500007C0489B05C0489B03C0489B01C09EC084
:10056000DF93C091AB02DD27CE54DD4F489B02C024
:10057000DF91EBCF2F930F931F9309B12FEF00FB68
:1005800020F94F933F9319B14FEF012700FB21F959
:100590003BE031C04E7F012F19B1216028C0102FE0
:1005A0004D7F2260000009B129C04B7F2460012FDC
:1005B000000019B12BC019B1477F28602AC04F7EB7
:1005C00009B120612CC04F7D19B120622FC04F7B33
:1005D00009B1206432C0422709B149934FEF0000AE
:1005E000102710FB20F919B11570A9F1297F91F29C
:1005F000012700FB21F909B1237F89F23150F0F185
:10060000102710FB22F919B1277E79F2012700FB90
:1006100023F92F7C81F209B1102710FB24F92F79DF
:1006200071F200C019B1012700FB25F92F7359F2AF
:1006300000C009B1102710FB26F9223040F200C09B
:1006400019B1012700FB27F9243028F64F772068DD
:1006500019B10000F9CF3B503195333011E01CBB8C
:10066000B8F0C31BD0400881033C41F10B3431F199
:100670001981412F1F772091A902121731F40936F1
:1006800091F10D3279F0013E69F022272093B002FA
:100690003F914F911F910F912F91DF91CF91CFBF3C
:1006A000CF9118950093B0023F914F911F910F91F8
:1006B0002F91DF91CCB3C0FD46CFF0CF0091B002B7
:1006C000002331F31091AE021123A1F53430A2F1D1
:1006D0003093AE020093AA021091AB023BE0311BB3
:1006E0003093AB0229C00091AE0201301CF50AE53F
:1006F00047FD09C03091010134FD20C00093010184
:10070000C3E9D2E01FC03091020134FD17C000934D
:100710000201CEE9D2E016C0052710E00BB91FC0D8
:10072000052722C0052727C005272CC0052710E074
:100730000BB933C04AE503C042ED01C0432FC4E109
:10074000D0E032E01AB11560589A0BB11AB95F9334
:1007500055E020E820FF05270BB9279517951C3F8A
:10076000D8F620FF052727950BB917951C3FC0F633
:1007700020FF0527279517950BB91C3F98F620FFFA
:100780000527279517951C3F0BB970F600C04991B6
:1007900020FF05270BB9279517951C3F38F620FF3A
:1007A000052727950BB917951C3F38F520FF05271E
:1007B000279517950BB91C3F10F520FF05272795A6
:1007C00017951C3F0BB9E8F4242F3A9519F60A7FC8
:1007D0005F910BB900C01091AF02C651D04011F02B
:1007E0001093A90211E01CBB01601AB11A7F402FBF
:1007F0004A7F0BB91AB94BB94BCF0527D3CF052781
:10080000D8CF0527DDCFFC018081807641F581813D
:10081000863029F583818230D1F0823269F08130CF
:10082000F1F480913D0290913E029093AD0280934D
:10083000AC0280913F02089580913A0290913B0270
:100840009093AD028093AC0280913C02089589E3BD
:1008500091E09093AD028093AC0282E2089580E033
:100860000895DC0120E532E03093AD022093AC0224
:100870008C918076803209F041C011968C9111974D
:10088000823081F08A30F1F08130C1F5E091400290
:10089000F09141020088F189E02DC90112966C9116
:1008A0000995089512969C91892F8150883030F5D2
:1008B000892F90E0895B9D4F9093AD028093AC02AD
:1008C00081E008951296EC911297EE2359F4E8E432
:1008D000F2E013968C911397819382E0E035F8074C
:1008E000C1F70CC08E2F8150883040F4F0E0E95BF6
:1008F000FD4F13968C91808380E0089580E00895E9
:100900006F927F928F929F92AF92BF92CF92DF921F
:10091000EF92FF920F931F93DF93CF93CDB7DEB784
:10092000AA970FB6F894DEBF0FBECDBF88E0FE01D8
:100930003196DF01982F1D929A95E9F7E8E4F2E0ED
:10094000DF011D928A95E9F7209A84B1897F84B9E5
:1009500085B1866085B9289880E395E70197F1F71E
:1009600083B190E08670907095958795823091055F
:1009700009F43FC08330910509F43DC0019709F1A6
:10098000CDD6FC0190934102809340020284F3850E
:10099000E02D0995882309F452C0DE011996EFE98C
:1009A000F1E082E201900D928150E1F7A3E0B1E025
:1009B000FE01399682E201900D928150E1F74FD805
:1009C0003AC04FD79093410280934002DE011996BE
:1009D000EDE7F1E082E201900D928150E1F7A3E0B2
:1009E000B1E0FE01399682E201900D928150E1F76B
:1009F00026C034D420C055D1FC019093410280938D
:100A000040020284F385E02D0995EFD18823B9F0E7
:100A1000DE011996EBE5F1E082E201900D92815042
:100A2000E1F7A3E0B1E0FE01399682E201900D9278
:100A30008150E1F79BD39093410280934002E09173
:100A40004002F09141028481958190933B02809312
:100A50003A02828180933C0280859185009731F033
:100A600090933E0280933D02868107C087E391E028
:100A700090933E0280933D0283D680933F02809103
:100A80003C028093520117B88FEF88B988EF8BB979
:100A900085E08AB91AB885BD82E08093B00087E00E
:100AA0008093B10084EC8093B30083B7817F83BFD0
:100AB000E0914002F09141020284F385E02D099516
:100AC000E1DB7894FF2411E0662463944E010894DE
:100AD000811C911C21E0C22ED12C94E0792E8CE255
:100AE000A82E81E0B82E02C0FF2410E0A895D4DB28
:100AF000112341F0E0914002F09141020484F58518
:100B0000E02D0995B89B27C067BA409140025091EB
:100B10004102D40120E030E018C0F901E85BFD4F4C
:100B2000E081EE2379F08C91853018F085508C931C
:100B300009C0EC93C601022E02C0880F991F0A94C7
:100B4000E2F7F82A2F5F3F4F1196FA0180819181D9
:100B50002817390714F3BA9B31C077BA83B781607D
:100B600083BF889583B78E7F83BFC5010197F1F757
:100B7000E0914002F09141020484F585E02D099551
:100B800000E010E012C00684F785E02D802F8F5F13
:100B90000995882341F0C601002E02C0880F991FD5
:100BA0000A94E2F7F82A0F5F1F4FE0914002F0919C
:100BB000410280819181081719072CF3FF2009F465
:100BC00094CF00E010E0EF2CFF24E7FCF09422C06B
:100BD000C701002E02C0959587950A94E2F780FF21
:100BE00017C08091020184FF13C0602F6F5F0088DF
:100BF000F189E02D82E492E00995682F82E492E089
:100C00005FDC02C049DBA8958091020184FFFACF26
:100C10000F5F1F4FE0914002F0914102808191816E
:100C200008171907ACF260CF449A80E38A95F1F770
:100C3000449880E090E030E048E1242F2A95F1F7D5
:100C40004598330F339B3160242F2A95F1F7459A4D
:100C500001968830910589F73093570280E090E043
:100C600048E1242F2A95F1F745983695339B306853
:100C7000242F2A95F1F7459A01968830910589F736
:100C80003093580208951F931FB7F8943C9A3D9AE9
:100C90003B98439A459A4498C7DF1FBF80E01F9155
:100CA00008958AE590E09093C6018093C50181EC98
:100CB00091E00895FC01009709F453C0A0915702F8
:100CC00080915802682F70E0CB01807F9070803F48
:100CD000910521F481E08093560202C010925602E1
:100CE0004A2F50E0A0FD03C020E830E002C02FEF03
:100CF00030E041FF02C020E030E042FD03C080E868
:100D000090E002C08FEF90E043FF02C080E090E0EF
:100D100020838183CA018074907025E09595879522
:100D20002A95E1F79A0120723070B3E03595279546
:100D3000BA95E1F7982F922BAA1FAA27AA1F9A2BE0
:100D40004071507055954795942B9283809156022F
:100D5000882339F484E0660F771F8A95E1F7962B94
:100D60009283809157029091580290935A028093F7
:100D7000590283E008958091D3019091D401892B89
:100D800031F01092D4011092D30181E0089587E5EB
:100D900092E069E572E042E050E0DFD60895FC01A0
:100DA000449A80E38A95F1F7449890E028E1822FF5
:100DB0008A95F1F74598822F8A95F1F7459A9F5FBA
:100DC0009830A9F7908120E038E1832F8A95F1F7D8
:100DD0004598990F339B9160832F8A95F1F7459A37
:100DE0002F5F283091F790830895DF93CF930F9270
:100DF000CDB7DEB7CE010196D2DF90E089818F704A
:100E0000813009F491E0892F0F90CF91DF910895FF
:100E10006F927F928F929F92AF92BF92CF92DF920A
:100E2000EF92FF920F931F93DF93CF930F92CDB763
:100E3000DEB773E0E72EF12CE822F92206E010E09D
:100E40004E010894811C911C68EBA62E6BE0B62E17
:100E500054E0752E40E3642E30E8C32E3BEBD32ED6
:100E6000C4019DDF898190E08073907024E09595A6
:100E700087952A95E1F78E159F0529F4F092640273
:100E8000E09263021CC0C5010197F1F780E090E099
:100E9000449A272D2A95F1F74598459A272D2A95AA
:100EA000F1F74498262D2A95F1F701968F31910597
:100EB00079F7C6010197F1F70150104089F60F90BC
:100EC000CF91DF911F910F91FF90EF90DF90CF9026
:100ED000BF90AF909F908F907F906F900895DF9319
:100EE000CF930F92CDB7DEB7CE01019658DF29819F
:100EF000822F8F70813079F580916102909162022A
:100F0000892B71F52295269526952370822F90E0E6
:100F10008130910571F0823091051CF4892B79F0B4
:100F200013C08230910541F0039771F480E090E0A6
:100F30000AC081E090E007C082E090E069DF809124
:100F400063029091640264DFCE01019628DF8981FB
:100F50008F70813029F0109262021092610256C0A7
:100F600081E090E090936202809361028981809396
:100F7000650280E797E10197F1F78CED95E0019725
:100F8000F1F780E090E050E030E2232F2A95F1F76E
:100F90004598550F339B51600000459A0196883063
:100FA000910599F780E090E030E040E2242F2A9507
:100FB000F1F74598330F339B31600000459A019655
:100FC0008830910599F7232F2F77452F4F7737FDDD
:100FD000219557FD4195332727FD309580915B0280
:100FE00090915C02820F931F90935C0280935B024E
:100FF000242F332727FD309580915D0290915E026A
:10100000820F931F90935E0280935D020F90CF91A9
:10101000DF9108953C9A3D9A3B98439A459A4498AB
:101020005EDF80916502829586958695837090E05B
:101030008130910571F0823091051CF4892B31F0DB
:101040000EC08230910541F0039749F480E090E0B2
:1010500005C081E090E002C082E090E0D9DE80E04F
:1010600008958091E7019091E801892B29F0109271
:10107000E8011092E7011DC090916502809166021F
:101080009817B9F420915B0230915C02809167025D
:10109000909168022817390761F440E020915D02C1
:1010A00030915E028091690290916A022817390797
:1010B00009F041E0842F0895FC01009709F454C021
:1010C00080915F0290916002892B41F01082118221
:1010D00012821092600210925F0246C0A0916502D7
:1010E0008A2F8295869586958370808360915B02B6
:1010F00070915C028FEF6138780714F481E806C0C4
:101100006038710514F08FE701C0862F40915D02B1
:1011100050915E029FEF4138590714F421E806C050
:101120004038510514F02FE701C0242F818322831A
:10113000992787FD909590936802809367023327E3
:1011400027FD309530936A0220936902A0936602CE
:10115000681B790B70935C0260935B02421B530B1C
:1011600050935E0240935D0283E0089585E890E02D
:101170009093DA018093D90187EB90E09093DE01A0
:101180008093DD0185ED91E008953C9A3D9A3B986E
:10119000439A459A449880E00895449A80E38A955A
:1011A000F1F7449880E090E030E048E1242F2A9560
:1011B000F1F74598330F339B3160242F2A95F1F7CF
:1011C000459A01968830910589F730936B0208950E
:1011D00080916B0290916C02891B0895FC0100972D
:1011E000B9F160916B02462F50E060FD03C020E82A
:1011F00030E002C02FEF30E041FF02C020E030E0DD
:1012000042FD03C080E890E002C08FEF90E043FF12
:1012100002C080E090E0208381839A0120743070C6
:1012200075E0359527957A95E1F7CA01807290703F
:1012300033E0959587953A95E1F7282B661F662749
:10124000661F262B4071507055954795242B22839D
:1012500080916B0280936C0283E0089589EC90E0AA
:101260009093EE018093ED018AEF90E09093F2016C
:101270008093F10189EE91E0089526B163B130E0E9
:10128000A90140715070A3E055954795AA95E1F7E3
:10129000C9018870907095958795482B862F80722C
:1012A000482BC90184709070880F991F482BC90181
:1012B0008270907073E0880F991F7A95E1F7482B40
:1012C0002072307055E0359527955A95E1F7422BFD
:1012D00080910F02843011F0842F0895862F90E0C2
:1012E00080719070880F991F880F991F842B089523
:1012F000DF92EF92FF920F931F93CF93DF93EC0156
:10130000409A00E5802F8A95F1F7B7DFD82E8091BB
:101310000F02823028F4D8828FEF89838A8329C014
:101320004098802F8A95F1F7A8DFF82E409A802FF9
:101330008A95F1F74098802F8A95F1F79EDFE82E85
:10134000409A802F8A95F1F74098802F8A95F1F77F
:1013500094DF182F409A802F8A95F1F78EDF4098FE
:10136000902F9A95F1F7409AD882F9828A83EB827E
:101370001C83DF91CF911F910F91FF90EF90DF9031
:101380000895DF92EF92FF920F931F93CF93DF9315
:1013900000E010E0C0E0D0E0EE24FF24B8E2DB2E55
:1013A0006CDF85FF04C00894E11CF11C01C021968C
:1013B0008D2D8A95F1F70F5F1F4F0436110581F7C8
:1013C000A2971CF420E030E009C080E090E022E227
:1013D000E216F10414F081E090E09C01C901DF9174
:1013E000CF911F910F91FF90EF90DF9008957F9222
:1013F0008F929F92AF92BF92CF92DF92EF92FF9225
:101400000F931F93DF93CF9300D000D00F92CDB7EF
:10141000DEB710910F02143009F07FC010916D02F9
:1014200010FD07C0CC24DD24E1E0F0E0AA24BB24B9
:1014300008C021E0C22ED12CE0E0F0E091E0A92E1E
:10144000B12CE159FD4F80E880831092710215DFC5
:10145000282F30E084FD05C0809171028160809367
:101460007102C9018074907011FF10C0892B29F49A
:1014700080917102826080937102EE24FF2484E0E7
:10148000782E08EF802E18E0912E44C0892BA9F702
:10149000809171028160EFCFF0DE85FD08C0972D4D
:1014A0009A95F1F70F5F1F4F04361105A9F785FFD5
:1014B00026C0E3DE182F892D8A95F1F7DEDE85FF41
:1014C00021C0882D8A95F1F7D8DE85FD1BC0012F3C
:1014D0000295007FD2DE182F1F70892D8A95F1F7B3
:1014E000CCDE85FD0FC0802F812BAB2809F08095C5
:1014F0002FE632E0C20ED31EF60180837CC0882D19
:101500008A95F1F70894E11CF11CF4E0EF16F10460
:1015100009F471C000E010E0BFCFCE010196E8DE13
:10152000998190958A8180958A836B81609590FDE1
:1015300003C040E850E002C040E050E091FF02C02C
:101540004FEF50E092FD03C020E830E002C020E001
:1015500030E093FF02C02FEF30E020936F02409302
:101560007002109271021230D0F18A81282F84FF0C
:1015700003C081E08093710294FF05C080917102E5
:1015800082608093710295FF05C080917102846032
:101590008093710225FF05C080917102886080935D
:1015A0007102133041F5962F62FF05C080917102E0
:1015B00080618093710291FF05C080917102806209
:1015C0008093710290FF05C08091710280648093C6
:1015D000710293FF10C08091710280680AC094FF6D
:1015E00003C081E08093710295FF05C08091710274
:1015F0008260809371020F900F900F900F900F9068
:10160000CF91DF911F910F91FF90EF90DF90CF90DE
:10161000BF90AF909F908F907F9008951F93DF931E
:10162000CF9300D000D00F92CDB7DEB71FB7F8949C
:10163000219A299884B18F7C84B985B1806385B95A
:10164000389A409A87B1817C87B988B18E6388B90E
:1016500088EE93E02CE231E0F9013197F1F7019740
:10166000D9F78FDE892B29F184E080930F0282E085
:1016700090E090936E0280936D02B9DE10926E023C
:1016800010926D0280917102282F80FF06C081E0C8
:1016900090E090936E0280936D0221FF34C08091A0
:1016A0006D0290916E02826090936E0280936D0243
:1016B0002AC0CE0101961CDE81E080930F02898151
:1016C00090E08F7090708330910519F41FBF8FEFF9
:1016D0001CC00F9789F48A818F70833069F48C81E4
:1016E0008F70833021F48D818F70833011F083E00F
:1016F00001C082E080930F028A8185FD03C083E0F0
:1017000080930F0274DE1FBF80E00F900F900F9048
:101710000F900F90CF91DF911F9108958CE091E091
:10172000909300028093FF018BEF91E00895009762
:1017300041F0DC01EFE6F2E083E001900D92815090
:10174000E1F7A2E7B2E0EFE6F2E083E001900D926C
:101750008150E1F783E0089580910D0290910E028F
:10176000892B31F010920E0210920D0281E0089543
:101770008FE692E062E772E043E050E0EED1089538
:1017800082E190E00895409888EB9BE0FC0131975E
:10179000F1F7419AFC013197F1F726B14198019791
:1017A000F1F786B1409A90E08C739070880F991F82
:1017B000880F991F30E02C7330703595279535953B
:1017C0002795822B8095982F83FD03C040E850E039
:1017D00002C040E050E091FF02C04FEF50E090FDAA
:1017E00003C020E830E002C020E030E092FF02C0F9
:1017F0002FEF30E02093750240937602109277022B
:1018000087FF03C081E08093770296FF05C0809137
:10181000770282608093770295FF05C080917702FE
:1018200084608093770294FF05C08091770288607E
:101830008093770208951F931FB7F894219A2998EF
:1018400087B1837C87B988B18C6388B988B183609C
:1018500088B987B1836087B996DF1FBF80E01F9189
:1018600008958BE591E0909315028093140289E42A
:1018700091E0909319028093180280E192E008951C
:10188000009741F0DC01E5E7F2E083E001900D9282
:101890008150E1F7A8E7B2E0E5E7F2E083E00190EC
:1018A0000D928150E1F783E008958091220290919A
:1018B0002302892B31F0109223021092220281E040
:1018C000089585E792E068E772E043E050E045D193
:1018D00008958FB7F894219A2998259A2D9A389AC5
:1018E000409A97B1917C97B998B19E6398B98FBF90
:1018F00080E008958F929F92AF92BF92CF92DF9235
:10190000EF92FF920F931F93DF93CF93CDB7DEB784
:1019100062970FB6F894DEBF0FBECDBF40988CE241
:1019200091E00197F1F760E070E08E010F5F1F4FCB
:101930009FE0F92EACE2B1E060FF04C02D9A319B2C
:10194000FECF03C02D983199FECF46B150E09A01E9
:101950002870307035952795CA0180719070F3E03A
:1019600095958795FA95E1F7282BCA0184709070B8
:10197000880F991F282B4072507035E05595479578
:101980003A95E1F7242BF801E60FF71F2F25208366
:10199000CD010197F1F76F5F7F4F6231710561F6FD
:1019A0002D9A409A89818F3009F046C08A818F3004
:1019B00009F042C093E0E92EF12CEC0EFD1E26E06A
:1019C00030E0CC24DD244E010894811C911C87E07A
:1019D000A82EB12CAC0EBD1ED7018C918E3019F003
:1019E0008F3021F406C063E070E005C060E070E075
:1019F00002C062E070E08401020F131FF601E55897
:101A0000FD4F40E050E006C0D8018D918D018193DB
:101A10004F5F5F4FDA01A20FB31F46175707A4F3BA
:101A20000894E11CF11CE3E0F0E0CE0EDF1EEA14A6
:101A3000FB0411F09D01D0CF62960FB6F894DEBF83
:101A40000FBECDBFCF91DF911F910F91FF90EF900F
:101A5000DF90CF90BF90AF909F908F90089586E8D1
:101A600091E090932902809328028AE392E0909378
:101A70002D0280932C0284E292E008950F931F932D
:101A8000CF93DF938C01662311F480E046C0862F4C
:101A9000992787FD909501979C01220F331F280FEE
:101AA000391FE901C558DD4FD901A957BD4FFE01C6
:101AB00083E001900D928150E1F7888180FD03C0A1
:101AC00040E850E002C040E050E081FF02C04FEF2C
:101AD00050E082FD03C020E830E002C020E030E0AA
:101AE00083FF02C02FEF30E0898190E080FD92E01B
:101AF00081FD946082FD916083FD98608A8180FD04
:101B0000906481FD906282FD906183FD9068F80190
:101B1000608321834283938384E0DF91CF911F917F
:101B20000F910895282F8091360290913702892BCA
:101B300031F0109237021092360281E00895215060
:101B400063E02602B0011124CB0185589D4F6957EF
:101B50007D4F43E050E001D00895FB01DC0104C05B
:101B60008D910190801921F441505040C8F7881B95
:081B7000990B0895F894FFCFD2
:101B7800FF5A5A36036500740020004D0061006B5F
:101B8800006F0054006F0020002800530029004E09
:101B980000450053002F0041007400610072006985
:101BA800005F0055005300420009022200010100B5
:101BB800803209040000010300000009210101002E
:101BC800012200000705810308000A360353004E6E
:101BD80000450053004D006F007500730065005FFD
:101BE8000074006F005F0055005300420036034E3A
:101BF80000650063002D0050006300200065006E42
:101C080000670069006E0065002000200020003693
:101C18000353006500670061004D0075006C007497
:101C28000069007400610070005F005500530042B5
:101C38000001002B0000000000000043061406BB52
:101C4800065A060100010032000000120000000AD6
:101C5800086F0731085C080100010031000000121C
:101C6800000000C508CD08E808EE0801002B0000B8
:101C780000000000000E0BF709AC0B970B010002E7
:101C880001002B000000120000001B0CC30B550CB8
:101C9800400C01000400B400000012000000690CB0
:081CA8007A0C920D3E0D0100C3
:00000001FF
